:100000009328FF3FFF3FFF3F0D1209008200493454
:100010004E34543452344F34443455345A344334C7
:100020004134203443344C34413456344534003464
:1000300050345534453444344534203450344134FC
:10004000533441345234003443344C344134563404
:100050004534203449344E3443344F3452345234CE
:1000600045344334543441340034433441344D3402
:10007000423449344F34203444344534003420343D
:1000800041344E34543449344734553441340034C7
:100090004E345534453456344134003456344534A6
:1000A000523449344634493451345534453400349B
:1000B0002034433441344D3442344934413444349F
:1000C000413400344C344134203443344C344134D2
:1000D00056344534203444344534423445340034B5
:1000E000543445344E34453452342034343420347E
:1000F000443449344734493454344F34533400344D
:1001000049344E34543445344E34543445344C34EC
:100110004F3400344434453420344E34553445345F
:1001200056344F340034860187018501831606302A
:100130009F00860105118510051085118512F0308C
:10014000870083120D120330A1004223422349236A
:1001500000305A230730272344305A231B232023FF
:10016000A600423C0319AE282608413C03192F295A
:100170002608433C031978292608443C0319AE2875
:100180002A304C231B232023A700423C03193A2981
:100190002708413C03192F292708433C03197829D4
:1001A0002708443C0319C2282A304C231B23202350
:1001B000A800423C031941292808413C03192F2972
:1001C0002808433C031978292808443C0319D628F9
:1001D0002A304C231B232023A900423C0319482921
:1001E0002908413C03192F292908433C0319782980
:1001F0002908443C0319EA282A304C231B232023D6
:10020000A200413C03190D292208423C03194F2941
:100210002208433C03197829FF2800308A22A602CD
:10022000031D2F2901308A22A702031D2F29023026
:100230008A22A802031D2F2903308A22A902031D46
:100240002F29492302305A23183027230330A100D5
:10025000851620305D23851210305D23A7280C30D1
:100260005323492324302723A10B37295629203033
:100270005D23A72844305A2320304C2344305A238E
:10028000AE2845305A2320304C2345305A23C2280B
:1002900046305A2320304C2346305A23D628473044
:1002A0005A2320304C2347305A23EA281E30A2001C
:1002B0000330A1000F30A3003030A4002030AA008A
:1002C000A30303196A2985156F2185116F21AA0BD4
:1002D00063295E2901305D23A20B5829A728230832
:1002E000A500A50B7129A40B6F293030A4000800CC
:1002F0004923353027231130272320305D2349231C
:10030000113027233F3027231B2344305A230A224E
:1003100000308A22A602031D002A01308A22A70289
:10032000031D002A02308A22A802031D002A03307E
:100330008A22A902031D002A0330A10049230230AA
:100340005A23483027231130272344305A231B23B4
:100350000A2226080319F629AB0027080319F629F3
:10036000AC0028080319F629AD0029080319F6295D
:10037000AE0049234E3027231130272344305A231F
:100380001B230A2226082B02031DEA2927082C0218
:10039000031DEA2928082D02031DEA2929082E0237
:1003A000031DEA2949231130272358302723260823
:1003B000AF00003094222708AF00013094222808B3
:1003C000AF00023094222908AF000330942220307D
:1003D0005D23A728492303305A2380302723433045
:1003E0005A238A30272320305D239E2949236230F7
:1003F000272340305A237030272320305D23A7283D
:10040000A1030319562949232430272320305D23D3
:100410001B23A728A601A701A801A9011B232023AC
:10042000A600423C03190E2A2608413C0319080085
:100430002608433C03190E2A2608443C03190E2AB9
:100440002A304C231B232023A700423C0319692A8E
:100450002708413C031908002708433C0319222AB6
:100460002708443C0319222A2A304C231B2320232B
:10047000A800423C0319712A2808413C03190800CE
:100480002808433C0319362A2808443C0319362A15
:100490002A304C231B232023A900423C0319792A2C
:1004A0002908413C0319882A2908433C03194A2A90
:1004B0002908443C03194A2A2A304C231B232023B1
:1004C000A200413C031908002208423C0319812A7A
:1004D0005F2A44305A2320304C2344305A23A7014A
:1004E0000E2A45305A2320304C2345305A23A80188
:1004F000222A46305A2320304C2346305A23A90161
:10050000362A47305A2320304C2347305A234A2A70
:10051000A9010800031783128D0083168C130C1495
:1005200083120C0803130800031783128D000313B2
:100530002F0803178C0083168C130C158B13553062
:100540008D00AA308D008C148B17831203130D1E9F
:10055000A72A831603170C11831203130D12080028
:100560000F30870000000708A20069230708A202D5
:10057000031DB02A0F3C031DBE2A0F34071AC72AD9
:10058000871ADC2A071BF12A871B062B0F34013040
:1005900087000000071A3134023087000000071A74
:1005A0003234043087000000071A333408308700E3
:1005B0000000071A41340F34013087000000871A09
:1005C0003434023087000000871A35340430870045
:1005D0000000871A3634083087000000871A42343A
:1005E0000F34013087000000071B373402308700CA
:1005F0000000071B3834043087000000071B393423
:10060000083087000000071B43340F340130870097
:100610000000871B2A34023087000000871B30341B
:10062000043087000000871B233408308700000057
:10063000871B44340F34B0220F3C031908001B2BD6
:10064000B022A2000F3C0319202B22080800A000B2
:100650000620003E031908004C23A00A2008282B7E
:100660008316FF3086008312051505108514FF30B0
:100670008600861B392B051185108613831686018B
:1006800083120800383053230C3053230630532391
:100690000800013053230800051505148510860055
:1006A0000511302308000515051085108600051179
:1006B00030230800803853230800A300FF30A40033
:1006C000FF30A500A50B622BA40B602BA30B5E2BA8
:1006D0000800FF30A300A30B6B2B0800FF3FFF3F78
:1006E000FF3FFF3FFF3FFF3FFF3FFF3FFF3FFF3F1A
:1006F000FF3FFF3FFF3FFF3FFF3FFF3FFF3FFF3F0A
:10070000FF3FFF3FFF3FFF3FFF3FFF3FFF3FFF3FF9
:10071000FF3FFF3FFF3FFF3FFF3FFF3FFF3FFF3FE9
:02400E003A3F37
:104200003000300030003000FF00FF00FF00FF00F2
:10421000FF00FF00FF00FF00FF00FF00FF00FF00A6
:10422000FF00FF00FF00FF00FF00FF00FF00FF0096
:10423000FF00FF00FF00FF00FF00FF00FF00FF0086
:10424000FF00FF00FF00FF00FF00FF00FF00FF0076
:10425000FF00FF00FF00FF00FF00FF00FF00FF0066
:10426000FF00FF00FF00FF00FF00FF00FF00FF0056
:10427000FF00FF00FF00FF00FF00FF00FF00FF0046
:10428000FF00FF00FF00FF00FF00FF00FF00FF0036
:10429000FF00FF00FF00FF00FF00FF00FF00FF0026
:1042A000FF00FF00FF00FF00FF00FF00FF00FF0016
:1042B000FF00FF00FF00FF00FF00FF00FF00FF0006
:1042C000FF00FF00FF00FF00FF00FF00FF00FF00F6
:1042D000FF00FF00FF00FF00FF00FF00FF00FF00E6
:1042E000FF00FF00FF00FF00FF00FF00FF00FF00D6
:1042F000FF00FF00FF00FF00FF00FF00FF00FF00C6
:10430000FF00FF00FF00FF00FF00FF00FF00FF00B5
:10431000FF00FF00FF00FF00FF00FF00FF00FF00A5
:10432000FF00FF00FF00FF00FF00FF00FF00FF0095
:10433000FF00FF00FF00FF00FF00FF00FF00FF0085
:10434000FF00FF00FF00FF00FF00FF00FF00FF0075
:10435000FF00FF00FF00FF00FF00FF00FF00FF0065
:10436000FF00FF00FF00FF00FF00FF00FF00FF0055
:10437000FF00FF00FF00FF00FF00FF00FF00FF0045
:10438000FF00FF00FF00FF00FF00FF00FF00FF0035
:10439000FF00FF00FF00FF00FF00FF00FF00FF0025
:1043A000FF00FF00FF00FF00FF00FF00FF00FF0015
:1043B000FF00FF00FF00FF00FF00FF00FF00FF0005
:1043C000FF00FF00FF00FF00FF00FF00FF00FF00F5
:1043D000FF00FF00FF00FF00FF00FF00FF00FF00E5
:1043E000FF00FF00FF00FF00FF00FF00FF00FF00D5
:1043F000FF00FF00FF00FF00FF00FF00FF00FF00C5
:00000001FF
